:03000000023E605D
:0C3E600078FFE4F6D8FD758171023EA7E2
:101420000A53746172743A20004950436F6E6E65BE
:1014300063745245510A004950436F6E6E65637480
:10144000003E432C562C43432CC0E4E0EFF2E5F081
:1014500020D1E8EDEAEEEC49500A003E432C4D4124
:10146000432C25303262583A25303262583A2530C2
:101470003262583A25303262583A25303262583A50
:1014800025303262582C4D414320E0E4F0E5F10A6A
:10149000003E432C5645522C20332E3120EEF220B4
:1014A00025732025732CC2E5F0F1E8FF2049502078
:1014B000ECEEE4F3EBFF0A004A616E203239203291
:1014C0003030380031353A30343A3534003E432C30
:1014D0004C442C50524F473A2020202020202020DE
:1014E00020202020202020202020202020202020FC
:1014F00020202020202020202020202020202020EC
:1015000020202020202020202020202020202020DB
:10151000202020202020202020202020202CC4E05B
:10152000F2E020EFF0EEF8E8E2EAE828F4E0E9EB98
:10153000290A003E2A2C312CCEF1EDEEE2EDFBE53E
:1015400020EFE0F0E0ECE5F2F0FB20F1E5F2E5E27F
:10155000EEE3EE20E8EDF2E5F0F4E5E9F1E00A0073
:101560003E412C4130312C2562752E2562752E2589
:1015700062752E2562752C495020E0E4F0E5F120DB
:10158000E0E4E0EFF2E5F0E00A003E412C413032C9
:101590002C2562752E2562752E2562752E256275A5
:1015A0002C495020E0E4F0E5F120EEF1ED2E20F1A1
:1015B000E5F0E2E5F0E00A003E412C4130332C2515
:1015C00062752E2562752E2562752E2562752C4951
:1015D0005020E0E4F0E5F120F0E5E72E20F1E5F021
:1015E000E2E5F0E00A003E412C4130342C256275E2
:1015F0002E2562752E2562752E2562752CCCE0F1A4
:10160000EAE020F1E5F2E80A003E412C4130352CB9
:101610002562752E2562752E2562752E2562752C24
:10162000D8EBFEE70A003E532C4130362C2562757C
:101630002CC2F0E5ECFF20EEE6E8E42E20EAE2E83A
:10164000F2E0EDF6E8E820282A3130ECF1290A0032
:101650003E2A2C312CC4EEEF2E20EFE0F0E0ECE53A
:10166000F2F0FB20F1E5F2E5E2EEE3EE20E8EDF248
:10167000E5F0F4E5E9F1E00A003E422C5330312C6C
:101680002562752CC6E4E0F2FC20E7E0EFF0EEF115
:10169000E020F1EEE5E4E8EDE5EDE8FF20EEF220F4
:1016A000F1E5F0E2E5F0E00A003E422C5330322C46
:1016B0002562752CCEE1ECE5ED20F120F1E5F0E2BC
:1016C000E5F0EEEC20E1E5E720EAE2E8F2E0EDF615
:1016D000E8E90A003E422C5330332C2562752CCFAA
:1016E000E5F0E5E7E0EFF3F1EA20EFF0E820EFEED8
:1016F000F2E5F0E520F1E2FFE7E820F120F1E5F086
:10170000E2E5F0EEEC0A003E422C5330342C256228
:10171000752CCDE5F220EFE5F0E5E4E0F7E820E414
:10172000E8E0E3EDEEF1F2E8EAE820E220F1E5F0AE
:10173000E2E5F00A003E422C5330352C2562752C30
:10174000CAE0EDE0EB20F8E8F0EEEAEEE2E5F8E0E2
:10175000F2E5EBFCEDEEE3EE20EEE1ECE5EDE00A88
:10176000003E532C5330362C25303262582530320F
:101770006258253032625825303262582530326244
:101780005825303262582C4D414320E0E4F0E5F119
:1017900020F8E8F0EEEAEEE2E5F8E0F2E5EBFCED49
:1017A000EEE3EE20EEE1ECE5EDE00A003E454E44CE
:1017B0000A0044756D7058202020202030302030E1
:1017C0003120303220303320303420303520303654
:1017D000203037203038203039203041203042202E
:1017E00030432030442030452030460A003A003A49
:1017F00020000A0044756D704420202020203030E5
:101800002030312030322030332030342030352029
:1018100030362030372030382030392030412030E9
:10182000422030432030442030452030460A0045D5
:101830007272206B657900526420656570726F6DFD
:101840000A005264204D454D0A00526420436F64E3
:10185000650A0044656275674950204F4E0A00448E
:10186000656275674950204F46460A0044656275B7
:101870006755736572204F6E0A004465627567553F
:10188000736572204F46460A0044656275674D7362
:1018900067204F6E0A0044656275674D7367204F7D
:1018A00046460A00436F6E666967206C6F636B2162
:1018B0000A00577220656570726F6D0A00205361CF
:1018C000766520656570726F6D210A004572722021
:1018D0004D414321004C6F61643E3E002A003C4173
:1018E00030313D003C4130323D003C4130333D0021
:1018F0003C4130343D003C4130353D003C413036C8
:101900003D003C21003C5330313D003C5330323DE2
:10191000003C5330333D003C5330343D003C5330A9
:09192000353D003C5330363D001A
:0647BA00010B00010900E3
:10477900C2AFC28E438910758BFF758DB7D2ABD28C
:044789008ED2AF22FB
:03001B00023C9C08
:103C9C00C0E0C083C082C0D0C2AFC28E758BFF752E
:103CAC008DB720060675A61E75A6E10509D202E59C
:103CBC000B6002050BE50AD394014002150A050EB0
:103CCC00E50E540F7050D20EE50E543F701AD20010
:103CDC00907AF2E0601204F0E0D394B4400A908041
:103CEC00007480F0C2AF80FE907AEDE0600204F0C8
:103CFC00907569E0600214F0907AF3E0D39401407F
:103D0C0003E014F0300502050CE50DD39464400477
:103D1C00D2068002050DE508D3940140021508D2A5
:0C3D2C008ED2AFD0D0D082D083D0E03255
:1008A400C291C290D2B5C20B7D027C007F07124771
:1008B4000D8F26E526646060097D017F601246C5C0
:1008C400D20BE4FDFC7F0B12470D8F26E52630E6A4
:1008D400097D04E4FF1246E9D20B7D017C007F0709
:1008E40012470D8F26E5267008FD7FFF1246C5D2FC
:1008F4000B300B03126000C2AFC288C2A8C2AA7533
:1009040089001240F59077A6E0B4FA09A3E064CE1A
:1009140070030209A4E4F526749E2526F582E434C6
:1009240077F583E4F00526E526B443EC9077A674C6
:10093400FAF0A374CEF0A374CCF09077AC740AF000
:10094400E4A3F0A304F0A3F09077B17403F0A374CC
:10095400CCF09077A274FFF0A3F0A3F0E4A3F0909E
:1009640077BD7405F0E4F526E5262401FFE433FEA3
:10097400749E2526F582E43477F583E0FD12476002
:100984000526E526C3944340DFE4F5A775A61E7546
:10099400A6E1907FF0F0A3F09080007480F080FED8
:1009A400D2AF9077B17403F0A374CCF0E49077B035
:1009B400F0123998C2B51224E5C20612444E90775B
:1009C400BDE0C3940350037403F0D20BC20DC20CF8
:1009D400D293200B077E147F201236A9E49079DD90
:1009E400F0124779C2AFA37408F090771C7424F016
:1009F400E4A3F09077A6E090771EF09077A7E090BC
:100A0400771FF09077A8E0907720F09077A9E09096
:100A14007721F09077AAE0907722F09077ABE0907E
:100A24007723F0750A01E49079DFF0C207C208C2A7
:100A340009C20AD2AF75A70775A61E75A6E11246AC
:100A44009E200B19AF267E007D031237AAE4FF1205
:100A54003B527E777FDDE4FB7D011238A4907AF26D
:100A6400E060037401F0E4907569F0A37455F0A399
:100A74007481F0E4F50CE4F50D907569E0700312EF
:100A84001F7F907AF3E0B401119080007410F0E4B9
:100A9400907AF3F0D20BC20CC20D908008E0F526D8
:100AA40030E405D2077410F0E52630E508D2099049
:100AB40080087420F0E52630E608D2089080087497
:100AC40040F0E50CD394034023908002E4F090803E
:100AD40001F0908000F0E50CD39406400FE4F50C8F
:100AE400C2039079DFF0750A0112444E9080A0E0B1
:100AF40070031241739080B8E070031241ED90804E
:100B0400D0E070031242CC908000E07013300710E4
:100B14001235A5907799EFF0D39400400312002684
:100B2400908002E07006908000E06005D205020A21
:100B34007AC205E4F50C907569E06003020A7A3024
:100B44000912122F61907799EFF0D394004005E0D9
:100B5400FF12478D200803020CD9122DEC907799CF
:100B6400EFF07003020A7A9077DDE054BF247F70BF
:100B740003020C3C147003020C1424026003020CE4
:100B84006F200B077E147F291236A9300F792003BA
:100B9400769077B5E070069077B9E0605B907AE97B
:100BA400E0FF9077B5E0B50724907AEAE0FE90770D
:100BB400B6E0B50618907AEBE0FE9077B7E0B5069C
:100BC4000C907AECE0FE9077B8E06E602B9077B9E9
:100BD400E06F7033907AEAE0FF9077BAE0B50727C8
:100BE400907AEBE0FF9077BBE0B5071B907AECE0DE
:100BF400FF9077BCE0B5070F9079DF7401F0120025
:100C040021750A01020CD9907AE974FFF0020CD91B
:100C1400907AF2E060037401F0907AE1E0FF90775B
:100C2400DFE06F6003020CD9907AE1E004F0E4F5B0
:100C34000A9079DDF0020CD9300303020CD99077C5
:100C4400ACE07003020A7A1247C1D203E4F50A90B9
:100C540079DDF0907AED04F0E4907AE0F0A3F020EE
:100C64000B737E147F371236A9806A907AF2E060A3
:100C7400037401F03003529077DDE020E74B907766
:100C8400DFE0FF907AE0E0FE6F600D907AE8E070BC
:100C940007EE146F703F8013907AE0E004F09077D1
:100CA40099E0FFD39404400312453590746574822F
:100CB400F0A37401F09077DFE0907467F07E747FA6
:100CC400657D03124075020A7A300F0920030690ED
:100CD4007AE974FFF0200303020D8EE50A706B12AB
:100CE40045E6EF60207E787FDD9078DEE02404FD29
:100CF400124075907AE8E06003020A7A9077BDE0CA
:100D0400F50A020A7A907AEDE0D3943C403C907A5A
:100D1400E8E07036907AED04F090771BE0702B12C7
:100D240047A7E49078DDF0A37412F0907AE1E090A4
:100D340078DFF0A374FDF090756C63A2019078E104
:100D440063A2017F121227C5809B12479CEF601596
:100D54009074657483F0E4A3F07E747F657D021261
:100D64004075020A7AE50A64016003020A7A9079FE
:100D7400DDE004F0E0C394055003020CE9C203E48F
:100D84009079DFF0120021020A7AE50A6401600317
:100D9400020A7A9079DFE014604624FE60421470FF
:100DA40003020E7C24046003020A7AE4F50C200F8B
:100DB400139079DF7404F09079DDE05401F0750A42
:100DC40001020A7A9080027410F0E49079DFF090C6
:100DD40079DD04F0750AC8907AE974FFF0020A7AA2
:100DE400907AE9E07003020E6B9078DD7480F090E5
:100DF40078DF7401F0E4A3F0A304F0A37430F0A34B
:100E0400747BF0E4F52674E42526F582E43478F561
:100E140083747DF074E52526F582E43478F583E463
:100E2400F0E52624079078DEF07C7A7DE99077B1AE
:100E3400E0FAA3E0FB7F02123F717E787FDDE526B6
:100E44002409FD124075907AE8E0601B1247C1D274
:100E540003E4F50A9079DDF0907AED04F0E4907AF9
:100E6400E0F0A3F0020A7A9079DF7404F09077BD81
:100E7400E02432F50A020A7A9080027410F0750AAE
:100E8400039079DDE06401FFF09079DF7401F0EF05
:100E940070199077B9E06013FCA3E0FDA3E0FEA312
:100EA400E0FF907AE912239B020A7A9077B5E0FC7E
:100EB400A3E0FDA3E0FEA3E0FF907AE912239B02E6
:040EC4000A7A80FE28
:010EC8002207
:100026009077DEE0B444047F0180027F009077DDA4
:10003600E0B447047E0180027E00EE5F604A90775E
:10004600A6E09077DFF09077A7E09077E0F09077E2
:10005600A8E09077E1F09077A9E09077E2F09077CA
:10006600AAE09077E3F09077ABE09077E4F09077B2
:10007600DE7452F090771563A2019080A863A20106
:100086007F061227C502089A907799E0C394085014
:10009600030208A39077A6E0FF9077DFE06F600386
:1000A6000208A39077A7E0FF9077E0E06F60030275
:1000B60008A39077A8E0FF9077E1E06F600302085D
:1000C600A39077A9E0FF9077E2E06F60030208A3B0
:1000D6009077AAE0FF9077E3E06F60030208A390B1
:1000E60077ABE0FF9077E4E06F60030208A39077B8
:1000F600DEE0B44415907715E0B4FF0E63A20190DC
:1001060080A863A2017F061227C5907AF2E06003F9
:100116007401F0907AF37464F09077DE7452F09084
:1001260077DDE0646D60030202A37BFF7A147941F8
:1001360012198B7BFF7A14795B9077A6E0F52FA3D3
:10014600E0F530A3E0F531A3E0F532A3E0F533A303
:10015600E0F53412198B752FFF7530147531B875AB
:1001660032FF7533147534C47BFF7A1479911219F2
:100176008B7BFF7A1479CD12198B7BFF7A15793335
:1001860012198B7BFF7A1579609077ACE0F52FA377
:10019600E0F530A3E0F531A3E0F53212198B7BFFD1
:1001A6007A15798A9077B5E0F52FA3E0F530A3E0CC
:1001B600F531A3E0F53212198B7BFF7A1579B890E9
:1001C60077B9E0F52FA3E0F530A3E0F531A3E0F52C
:1001D6003212198B7BFF7A1579E69077A2E0F52F1C
:1001E600A3E0F530A3E0F531A3E0F53212198B7BDD
:1001F600FF7A16790990779EE0F52FA3E0F530A3F4
:10020600E0F531A3E0F53212198B7BFF7A167926D9
:100216009077BDE0F52F12198B7BFF7A1679501275
:10022600198B7BFF7A167979A20FE433F52F121911
:100236008B7BFF7A1679A9907AE8E0F52F12198B55
:100246007BFF7A1679D4907AF2E0F52F12198B7B20
:10025600FF7A17790790771BE0F52F12198B7BFF32
:100266007A177935A201E433F52F12198B7BFF7AC1
:10027600177961907AE2E0F52FA3E0F530A3E0F577
:1002860031A3E0F532A3E0F533A3E0F53412198B80
:10029600123A7E7BFF7A1779AC12198B229077DDA2
:1002A600E0644C70757E177FB21236A99077E5E050
:1002B600F527A3E0F528E4F52A7E177FED1236A987
:1002C6007D03AF28AE271237AA7E177FEF1236A915
:1002D600E4F529852882852783E0FF74E72529F53B
:1002E60082E43477F583EFF00528E52870020527C8
:1002F6000529E529B410DC7E777FE7E4FB7D101243
:1003060038A47E177FF21236A9052AE52AC394106F
:1003160040A77E177FF21236A9229077DDE0646C43
:10032600705CF52B7E177FF41236A9E4F52AAF2B05
:100336007E007D031237AA7E177FEF1236A9E4F5F9
:1003460029A82BE6FF74E72529F582E43477F5839F
:10035600EFF0052B0529E529B410E67E777FE7E463
:10036600FB7D101238A47E177FF21236A9052AE506
:100376002AC3940840B87E177FF21236A9229077D6
:10038600DDE0644B7061F52974CF2529F582E434EC
:1003960077F583E0603274CF2529F582E43477F56A
:1003A60083E0F4602374CF2529F582E43477F5835E
:1003B600E0FF74E52529F582E43477F583E0B50797
:1003C600100529E529B408C09075697432F0020851
:1003D6009A9077DD7421F0300B0302089A7E187F1D
:1003E6002F1236A902089A9077DDE0B4521A200B34
:1003F600077E187F371236A99077DD7472F07E7704
:100406007FDD7D08123FF5229077DDE06449704577
:10041600200B077E187F421236A99077E5E0F52774
:10042600A3E0F528E4F529852882852783E0FF7473
:10043600E72529F582E43477F583EFF00528E528EA
:10044600700205270529E529B480DC7E777FDD7DEE
:100456008A123FF5229077DDE064437079A3E06469
:10046600527046200B077E187F4A1236A99077E510
:10047600E0F527A3E0F528E4F5298528828527837A
:10048600E493FF74E72529F582E43477F583EFF0EA
:100496000528E528700205270529E529B480DB7EB5
:1004A600777FDD7D8A123FF5229077DEE064576024
:1004B600030208A39077E5E0F527A3E0F52874E7A3
:1004C6002529F582E43477AD82FC7B80AF28AE2700
:1004D6001245B202089A9077DDE064446003020593
:1004E6006D9077E5E0FF6444700302089AEFB4313B
:1004F6000CC20B7E187F531236A902089A9077E534
:10050600E0B4300CD20B7E187F5F1236A902089A2F
:100516009077E5E0B4320CD20C7E187F6C1236A9C7
:1005260002089A9077E5E0B4330CC20C7E187F7A05
:100536001236A902089A9077E5E0B4340CD20D7E03
:10054600187F891236A902089A9077E5E0B4350C2F
:10055600C20D7E187F961236A902089A9077E5E0BA
:10056600FF12001E02089A907569E07013200B07AF
:100576007E187FA41236A99077DD7421F002089ABE
:100586009075697432F09077DDE0FFB4510A90807F
:10059600007480F0C2AF80FEEF64577045200B07F1
:1005A6007E187FB21236A99077E6E0907799F0E44C
:1005B600F529907799E0FFE529C39F400302089A41
:1005C60074E72529F582E43477F583E0FF9077E533
:1005D600E025292414F582E43476F583EFF0052925
:1005E60080D09077DDE06453600302069C200B0701
:1005F6007E187FBD1236A99077A6E0FF90761DE0A3
:100606006F703C9077A7E0FF90761EE06F70309099
:1006160077A8E0FF90761FE0B507249077A9E0FF62
:10062600907620E0B507189077AAE0FF907621E053
:10063600B5070C9077ABE0FF907622E06F601690DE
:1006460077DD7421F0300B0302089A7E187FCC12F6
:1006560036A902089AE4F529E4F50DAF29FE7414CB
:100666002529F582E43476F583E0FD1247600529F5
:10067600E529C394FE40E19080007480F0C2AFE4A7
:10068600907FF0F0A3F0907FFD74AAF0A374FFF0C2
:10069600A37455F080FE9077DDE0644F704C907740
:1006A600E5E0F527A3E0F528E5284527700A200BA5
:1006B600077E187FD51236A9200B077E187FDC121D
:1006C60036A9E4F52974E72529F582E43477F5831C
:1006D600E0852882852783F00528E528700205270E
:1006E6000529E529B480DE02089A9077DDE0FFB49B
:1006F60045279080007480F09077E5E0FDA3E090B8
:100706007FF0CDF0A3EDF0C2AF907FFD74AAF0A309
:1007160074FFF0A37455F080FEEF64656003020871
:100726009A9077E5E0FFA3E0907FF0CFF0A3EFF09B
:10073600E4F527F528D3907FF1E09528907FF0E047
:1007460095274020E4F50D2528FFE5273401FE8591
:100756002882852783E0FD1247600528E528700278
:10076600052780D17E187FDE123EECEF4E60201208
:1007760000039077ACEFF01200039077ADEFF01224
:1007860000039077AEEFF01200039077AFEFF07EA4
:10079600187FE4123EECEF4E60201200039077B50E
:1007A600EFF01200039077B6EFF01200039077B7E0
:1007B600EFF01200039077B8EFF07E187FEA123E52
:1007C600ECEF4E60201200039077B9EFF0120003B1
:1007D6009077BAEFF01200039077BBEFF0120003A8
:1007E6009077BCEFF07E187FF0123EECEF4E602063
:1007F6001200039077A2EFF01200039077A3EFF0B8
:100806001200039077A4EFF01200039077A5EFF0A3
:100816007E187FF6123EECEF4E60201200039077B2
:100826009EEFF012000390779FEFF012000390778F
:10083600A0EFF01200039077A1EFF07E187FFC1274
:100846003EECEF4E60081243F19077BDEFF0E4F511
:1008560029E4F50DE5292401FFE433FE749E2529DC
:10086600F582E43477F583E0FD1247600529E52932
:10087600C3944340DC9080007480F0C2AFE4907F64
:10088600F0F0A3F0907FFD74AAF0A374FFF0A374B8
:0D08960055F080FE7E777FDD7D08123FF576
:0108A3002232
:10457A00AE07EEC39430400BEED394395005EE24C7
:10458A00D0FF22EEC39461400BEED394665005EE41
:10459A0024A9FF22EEC39441400BEED39446500562
:0845AA00EE24C9FF22AF062236
:10474600907714E004F07006907713E004F0907709
:0A47560013E0FEA3E0FF12472A2241
:1000030012474612457AEFC454F0FEC00612474623
:0800130012457AD0E02FFF2214
:1043F100E4907C34F0124746907C35EFF0C3943062
:104401004018E0FFD394395011907C34E0246CF5CE
:1044110082E43475F583EFF08011907C34E0246CF4
:10442100F582E43475F583E4F0800C907C34E0048B
:10443100F0E0D3940840BE752F007530007531004F
:0C444100E4F5327B017A75796C122AAA2E
:01444D00224C
:043EEC008E2C8F2D5C
:103EF000907713E4F0A374FFF0124746EF606EF47E
:103F0000606B852D82852C83E493B507EC752E01BB
:103F1000E52D252EF582E4352CF583E4936025907C
:103F20007714E0252EFF907713E03400FE12472A25
:103F3000E52D252EF582E4352CF583E493B50704B1
:103F4000052E80CCE52D252EF582E4352CF583E475
:103F50009370A6E52E24FFFFE434FFFE907714E073
:103F60002FF0907713E03EF07E007F0122E4FEFF09
:013F7000222E
:103998007E197F02123EECEF4E70037F01227E19E2
:1039A8007F05123EECEF4E600C124746EF24D02400
:1039B800FF920F8002D20F7E197F0B123EECEF4E62
:1039C800600C124746EF24D0907AE8F08005E49026
:1039D8007AE8F07E197F11123EECEF4E600C124728
:1039E80046EF24D0907AF2F08005E4907AF2F07EE7
:1039F800197F17123EECEF4E600C124746EF24D0A9
:103A080090771BF08005E490771BF07E197F1D12DC
:103A18003EECEF4E600C124746EF24D024FF920193
:103A28008002C2019077A663A201907AE263A201A4
:103A38007F061227C530013B7E197F23123EECEF2B
:103A48004E6030120003907AE2EFF0120003907A91
:103A5800E3EFF0120003907AE4EFF0120003907A9B
:103A6800E5EFF0120003907AE6EFF0120003907A87
:063A7800E7EFF07F0022E1
:1044A7009079DEE0C3947C503D9079DEE0FE04F025
:1044B700741C2EF582E43477F583EFF0BF0A27905A
:1044C70079DEE0FF04F0741C2FF582E43477F5837E
:1044D700E4F09079DEE0FF123BFC9079DE7408F09F
:0744E70090771DE004F022B4
:10444E009080007480F090779E63A201F583F582D0
:10445E0063A2017F081227C59077A663A201908000
:10446E008863A2017F0A1227C5908092E4F0A3749C
:10447E0032F0A37401F09077B0E0FF9080B1F0902D
:10448E0080E1EFF09080957455F0A3F09080007469
:09449E0001F090800974F0F02295
:10417300908009E04410F09080A0E0706C9080A1E2
:104183007482F09080A874FFF0A3F0A3F0A3F07FF3
:10419300039080AEEFF07FCBA3EFF07F039080AC72
:1041A300EFF0A374CBF09080007402F0907C2612A1
:1041B30023A700000000907C26E0908040F0907CD4
:1041C30027E0908041F0907C28E0908042F0907C42
:1041D30029E0908043F0A3E4F0A3F0A3F0A3F090D0
:0941E3008018F0A3F0A3F0A3F092
:0141EC0022B0
:1042CC00908009E04440F09080D17482F09077B1F6
:1042DC00E0FF9080DEF09077B2E0FF9080DFF0900E
:1042EC0080027402F0907C2A1223A7000000009038
:1042FC007C2AE0908058F0907C2BE0908059F090D4
:10430C007C2CE090805AF0907C2DE090805BF0A3A8
:10431C00E4F0A3F0A3F0A3F0908030F0A3F0A3F0AE
:02432C00A3F0FC
:01432E00226C
:1041ED00908009E04420F09080B8E0706C9080B928
:1041FD007482F07F039080C6EFF07FCDA3EFF07F48
:10420D00039080C4EFF0A374CDF09080C074FFF0E4
:10421D00A3F0A3F0A3F09080017402F0907C2E1215
:10422D0023A700000000907C2EE090804CF0907C45
:10423D002FE090804DF0907C30E090804EF0907C9F
:10424D0031E090804FF0A3E4F0A3F0A3F0A3F09041
:09425D008024F0A3F0A3F0A3F00B
:014266002235
:103F71008C278D28A907EAFDE975F018A424ACFF68
:103F8100E5F034808F82F583EDF0EBFDE975F018F3
:103F9100A4FFAEF024ACFBEE34808B82F583A3ED5D
:103FA100F08528828C83E0FDEF24A8FFEE3480FEAB
:103FB1008F82F583EDF08528828C83A3E08F828E3A
:103FC10083A3F0852882852783A3A3E0FDE975F00B
:103FD10018A424A8FFE5F03480FE8F82F583A3A303
:103FE100EDF08528828C83A3A3A3E08F828E83A327
:043FF100A3A3F02274
:063FF5008D2CAB07AA06AB
:103FFB00908000E020E572907C26E0FCA3E0FDA31E
:10400B00E0FEA3E0F5308E2F8D2E8C2DAE02AF038C
:10401B008E838F8263A201E52F540744C0F58385FD
:10402B00308263A201AF2C122837E4FCFDFEE53091
:10403B00252CF530EE352FF52FED352EF52EEC35F5
:10404B002DF52D908040E52DF0A3E52EF0A3E52F67
:10405B00F0A3E530F09080007420F0AF30AE2FADC0
:09406B002EAC2D907C2612239B43
:014074002229
:064075008D27AB07AA062F
:10407B00908002E020E572907C2AE0FCA3E0FDA397
:10408B00E0FEA3E0F52B8E2A8D298C28AE02AF0320
:10409B008E838F8263A201E52A540744D0F5838572
:1040AB002B8263A201AF27122837E4FCFDFEE52B20
:1040BB002527F52BEE352AF52AED3529F529EC3593
:1040CB0028F528908058E528F0A3E529F0A3E52AE8
:1040DB00F0A3E52BF09080027420F0AF2BAE2AAD4D
:0940EB0029AC28907C2A12239BC9
:0140F40022A9
:023B52008F28BA
:103B5400908001E030E5037F0022907C2EE0FCA3FE
:103B6400E0FDA3E0FEA3E0F52C8E2B8D2A8C29909A
:103B74007AE263A201E52B540744C8F583852C82BD
:103B840063A2017F0612284DE52C2406F52CE435AA
:103B94002BF52BE4352AF52AE43529F5299079E02B
:103BA40063A201E52B540744C8F583852C8263A2E4
:103BB40001AF2812284DE4FCFDFEE52C2528F52C48
:103BC400EE352BF52BED352AF52AEC3529F5299020
:103BD400804CE529F0A3E52AF0A3E52BF0A3E52C1E
:103BE400F09080017420F0AF2CAE2BAD2AAC29905C
:073BF4007C2E12239BAF2879
:013BFB0022A7
:1035A5009081E0E0F527052705270527052705274D
:1035B50005270527052705270527908010E0F52A0B
:1035C500A3E0F52BA3E0F52CA3E0F52D9081E1E038
:1035D500F527052705270527052705270527052796
:1035E500052705270527908014E0F52EA3E0F52F84
:1035F500A3E0F530A3E0F531E530B52C08E531B5AC
:103605002D037F0022E4F527E530540744E0F583D8
:1036150085318263A2019077DD63A2017F081228BC
:103625007D9077DF63A20190771563A2017F061273
:1036350027C59077DDE0F528A3E0F529E4F5279087
:1036450077DDE0702AA3E024F8F527E53054074438
:10365500E0F58385318274082582F582E43583F5AA
:103665008363A2019077DD63A201AF2712287DAEA7
:1036750028E4FCFDE5312529F531E5303EF530ED51
:10368500352FF52FEC352EF52E908014E52EF0A371
:10369500E52FF0A3E530F0A3E531F090800074400C
:0336A500F0AF275C
:0136A80022FF
:102DEC009081E6E0F5270527052705270527052708
:102DFC0005270527052705270527908028E0F52AB4
:102E0C00A3E0F52BA3E0F52CA3E0F52D9081E7E0F2
:102E1C00F527052705270527052705270527052756
:102E2C0005270527052790802CE0F52EA3E0F52F2C
:102E3C00A3E0F530A3E0F531E4F527E530B52C0A35
:102E4C00E531B52D05C208022F46E530540744F094
:102E5C00F58385318263A2019077DD63A2017F083F
:102E6C0012287D9077DDE0F528A3E0F529E52945CA
:102E7C002870099080027410F07F0022907AE9E0AB
:102E8C00FFF4602D9077DFE06F7076907AEAE0FFC8
:102E9C009077E0E06F706A907AEBE0FF9077E1E07A
:102EAC006F705E907AECE0FF9077E2E06F602280CA
:102EBC00509077DFE0907AE9F09077E0E0907AEA52
:102ECC00F09077E1E0907AEBF09077E2E0907AEC9A
:102EDC00F09077DDE0702AA3E024F8F527E5305474
:102EEC000744F0F58385318274082582F582E43538
:102EFC0083F58363A2019077DD63A201AF271228CB
:102F0C007DAE28E4FCFDE5312529F531E5303EF5B3
:102F1C0030ED352FF52FEC352EF52EAF2DAE2CAD2B
:102F2C002BAC2AAB31AA30A92FA82ED312238A405E
:102F3C00099080027410F07F002290802CE52EF016
:102F4C00A3E52FF0A3E530F0A3E531F090800274F7
:042F5C0040F0AF276B
:012F6000224E
:102F61009081E3E0F5270527052705270527052794
:102F71000527052705270527052790801CE0F52A49
:102F8100A3E0F52BA3E0F52CA3E0F52D9081E4E07F
:102F9100F5270527052705270527052705270527E0
:102FA100052705270527908020E0F52EA3E0F52FC2
:102FB100A3E0F530A3E0F531E4F527E530B52C0ABF
:102FC100E531B52D05C2090230ACE530540744E8BE
:102FD100F58385318263A20190746963A2017F0E3A
:102FE100122893907469E0F528A3E0F52990747193
:102FF100E0FFF46045907AE2E0FEEF6E706EA3E0D0
:10300100FF907472E06F7064907AE4E0FF907473E3
:10301100E06F7058907AE5E0FF907474E06F704C47
:10302100907AE6E0FF907475E06F7040907AE7E087
:10303100FF907476E06F60048032D2D9907469E0B9
:10304100702AA3E024F2F527E530540744E8F5831C
:10305100853182740E2582F582E43583F58363A27E
:103061000190746963A201AF27122893AE28E4FC92
:10307100FDE5312529F531E5303EF530ED352FF50A
:103081002FEC352EF52EAF2DAE2CAD2BAC2AAB315E
:10309100AA30A92FA82ED312238A5006E529452844
:1030A10070099080017410F07F0022908020E52E3D
:1030B100F0A3E52FF0A3E530F0A3E531F090800116
:0530C1007440F0AF2790
:0130C60022E7
:0436A9008E2C8F2DA7
:1036AD00E4F52EF52F908000E030E511052FE52F84
:1036BD007002052ED394E8E52E940340E890800027
:1036CD00E030E5030237A9907C26E0FCA3E0FDA3E2
:1036DD00E0FEA3E0F5338E328D318C30E533FFE51E
:1036ED00325407FEE42FF52FEE34C0F52E852F82D0
:1036FD00F5837423F0052FE52F7002052E532EC789
:10370D00F582852E83740AF0052FE52F7002052EA4
:10371D00532EC79077A663A201852E83852F8263D2
:10372D00A2017F061228377406252FF52FE4352EBA
:10373D00F52E852C83852D8263A201852E83852F01
:10374D008263A20112281BE4FCFDFE907C26E0F8AA
:10375D00A3E0F9A3E0FAA3E02FFFEE3AFEED39FD69
:10376D00EC38FCEF2408FFE43EFEE43DFDE43CFCB8
:10377D00907C2612239B907C26E0908040F0907CDC
:10378D0027E0908041F0907C28E0908042F0907C82
:0C379D0029E0908043F09080007420F040
:0137A90022FD
:0638A4008E2C8F2D8D2EED
:1038AA00E4F52FF530908000E030E5110530E53081
:1038BA007002052FD394E8E52F940340E890800026
:1038CA00E030E503023997907C26E0FCA3E0FDA3F3
:1038DA00E0FEA3E0F5348E338D328C31E534FFE51A
:1038EA00335407FEE42FF530EE34C0F52F853082CD
:1038FA00F5837423F00530E5307002052F532FC786
:10390A00F582852F83EBF00530E5307002052F53E1
:10391A002FC79077A663A201852F8385308263A281
:10392A00017F0612283774062530F530E4352FF565
:10393A002F852C83852D8263A201852F8385308272
:10394A0063A201AF2E1228377408252EF52EFFE444
:10395A00FCFDFEE5342FF534EE3533F533ED353223
:10396A00F532EC3531F531908040E531F0A3E5329E
:10397A00F0A3E533F0A3E534F09080007420F0AFB3
:0D398A0034AE33AD32AC31907C2612239B5D
:01399700220D
:023BFC008F40F8
:103BFE00E4F541F542908000E030E5110542E542E2
:103C0E0070020541D394E8E541940340E8908000AA
:103C1E00E020E579907C26E0FCA3E0FDA3E0FEA386
:103C2E00E0F5468E458D448C43E546FFE545540749
:103C3E00FEE42FF542EE34C0F54190771C63A201ED
:103C4E0085418385428263A201AF40122837E4FC8E
:103C5E00FDFEE5462540F546EE3545F545ED354488
:103C6E00F544EC3543F543908040E543F0A3E5443D
:103C7E00F0A3E545F0A3E546F09080007420F0AF88
:0D3C8E0046AE45AD44AC43907C2612239B0E
:013C9B002206
:0637AA008E2C8F2DAB05F3
:1037B000E4F52EF52F908000E030E511052FE52F80
:1037C0007002052ED394E8E52E940340E890800023
:1037D000E030E5030238A3907C26E0FCA3E0FDA3E3
:1037E000E0FEA3E0F5338E328D318C30E533FFE51A
:1037F000325407FEE42FF52FEE34C0F52E852F82CC
:10380000F5837423F0052FE52F7002052E532EC784
:10381000F582852E83EBF0052FE52F7002052E90A3
:1038200077A663A201852E83852F8263A2017F067E
:103830001228377406252FF52FE4352EF52E532E3A
:10384000C7E52C852F82852E83F0052FE52F70028A
:10385000052E532EC7F582852E83E52DF0052FE525
:103860002F7002052E532EC7E533240AF533E435B5
:1038700032F532E43531F531E43530F530908040C1
:10388000E530F0A3E531F0A3E532F0A3E533F090A5
:1038900080007420F0AF33AE32AD31AC30907C2676
:0338A00012239B55
:0138A3002202
:10472A00E5D220E0FBC2AF438E2075D2028F828E83
:0B473A0083E0FFE4F5D2538EDFD2AF26
:014745002251
:10476000E5D220E0FBC2AF43D2028F828E83EDF010
:0947700075D25063D250D2AF2281
:1040F500E4FDED2401FFE433FE12472A749E2DF5FD
:1041050082E43477F583EFF00DBD3FE6E4FDED2461
:104115007FFFE433FE12472A74942DF582E434754B
:10412500F583EFF074942DF582E43475F583E07032
:104135001B74942DF582E43475F5837420F0749521
:104145002DF582E43475F583E4F080040DBD80BE61
:10415500E4907613F0FDEDFF7E0012472A74142DCE
:0D416500F582E43476F583EFF00DBDFEE940
:01417200222A
:0245B2008B2C50
:1045B400A2AF921EC2AF85A22D53A2FE8E838F821C
:1045C40005A28C838D8274091228C1E52C53A2FEA6
:1045D40043A2201228C353A2DF852DA2A21E92AFAC
:0145E400FFD7
:0145E50022B3
:10470D00A2AF921EC2AF8C838D82EF1228C143A23D
:0C471D00201228C353A2DFA21E92AFFF9F
:01472900226D
:0246C5008F273D
:1046C700A2AF921EC2AFE4F5838D8274061228C191
:1046D700E52743A2201228C353A2DFA21E92AF7F71
:0146E70001D1
:0146E80022AF
:0246E9008F2719
:1046EB00A2AF921EC2AFE4F5838D82740A1228C169
:1046FB00E52743A2201228C353A2DFA21E92AF7F4D
:01470B0001AC
:01470C00228A
:1026EA00A907E7FFA805EF93C3966008403B74FC6F
:1026FA002FFF80F00F08EF93C3966008402B74FBFE
:10270A002FFF80E00F08EF93C3966008401B74FA0E
:10271A002FFF80D00F08EF93D3966008400B74F90F
:10272A002FFF80C01F1F1F1F1FEF54FEF80303F760
:10273A00E893FC08E893FD08E893FE08E893FF2273
:10274A0009E993C39D6008402974FB29F980F109BE
:10275A00E993C39E6008401A74FA29F980E209E9EC
:10276A0093D39F6008400B74F929F980D31919197A
:10277A001919E9C313C313FF22740093F8ECC39821
:10278A004024701F740193F8EDC3984019701474B3
:0E279A000293F8EEC398400E7009740393F892
:1027A800EFC39840037F00227F0122EDF8E6F0088E
:1027B800A3DFFA22EDF8E0F608A3DFFA22E0A3632C
:1027C800A201F0A363A201DFF475A2002263A201B3
:1027D800F0A363A20122E0A363A201F0A363A20114
:1027E800E0A363A201F0A363A201E463A201F0A342
:1027F80063A201DFE175A20022E0A363A2016DFEDE
:10280800936CFDEE058393FC158363A201DFEA75E3
:10281800A200227F00E493A363A201F00F600CA33F
:10282800E583C2E3F58363A20180EA75A20022E092
:10283800A363A201F0A3E583C2E3F58363A201DFEA
:10284800EE75A20022E0A363A201F0A3E583C2E42F
:10285800D2E3F58363A201DFEC75A20022E0A36353
:10286800A201F0A3E58344F8C2E5F58363A201DF82
:10287800EC75A20022E583C2E3F583E0A363A2011D
:10288800F0A363A201DFEE75A20022E583C2E4D2C1
:0A289800E3F583E0A363A201F0A3BF
:1028A20063A201DFEC75A20022E58344F8F583E020
:1028B200A363A201F0A363A201DFEE75A20022F9D5
:1028C20022C002C004C00612FFF0D006D004D0021B
:0128D20022E3
:103DD2000A536572763A004572724C656E210A008A
:103DE200205544502054696D654750530A00200AFB
:103DF200444154414752414D3A20002043414E2014
:103E020054696D654750530A0020547261737353AD
:103E1200656E644552520A000ACEF8C4EBE8EDFB27
:103E220043414E210A000A45727241647243414E77
:103E32003A000A00205265496E69742043414E0AD5
:103E4200002043414E283029203E20544F210A00B1
:0E3E520020545520300A0020545520310A001B
:03001E00E4FF22DA
:10467600C2A9438902758C48758A4875D90475DBC9
:104686004875DC4875DD4875DE48E4F5E9F5F9D28C
:08469600D9C2DAD28CD2DE2277
:10464800C2D9907B08E07013E5E92419F5EB30D75F
:1046580006E5F904F5FB2285F9FB22E5E924C8F50E
:0E466800EB30D706E5F904F5FB2285F9FB22BD
:1044EE00C2D9907B08E0702C302B16E5E92432F50A
:1044FE00EB30D707E5F904F5FB800385F9FBC22BFA
:10450E0022E5E92405F5EB30D706E5F904F5FB22A3
:10451E0085F9FB22E5E92432F5EB30D706E5F904FF
:07452E00F5FB2285F9FB22D9
:10469E00124676907B08E0C394645006124267126D
:1046AE004648120022D22AE4F558907C20F0F547B5
:0746BE00F55CC22BF55A2246
:10453500EF24FCF547200B127E3D7FD21236A97E73
:10454500777FE1E4FBAD471238A4E547D3940D40EE
:1045550010200B077E3D7FD91236A9E4F547D228F6
:10456500229077E163A201907C1063A201AF47120C
:0545750027C5C2282249
:0F478D00D3EF6480948D5006E55C70028F5C2240
:101F7F0020D90302205C202A0302205CE55C60521A
:101F8F00907469540FFF7D491227BCE549640170B5
:101F9F001E907471E0B4FF0ED22C200B127E3D7F89
:101FAF00E21236A98009302C06E4F55C02205C129F
:101FBF00464812432F200B077E3D7FF01236A92093
:101FCF000B0B7E747F69E4FBAD5C1238A4E4F55C07
:101FDF00807BE5476043907C14E02405F527D3947C
:101FEF000D4007E4F547D2288063907C10E5275415
:101FFF000FFF7D491227BCE54930E702D22BE54997
:10200F00B40109302C06E54C6401600312432F1212
:10201F004648E4F547D2288034E559601E907AF49B
:10202F00540FFF7D491227BCE549B40103202C034F
:10203F0012432F124648E4F559801220100C907B62
:10204F0008E0C3946450031243911246481230C7FC
:10205F008F27EF70030221231244EEE4F55AE5496E
:10206F00B4010CD22C200B077E3D7FFD1236A9E563
:10207F005BC394C8502D30032AE549B4420DE54C9B
:10208F00B4020890771BE0640160187409255BF5B2
:10209F0082E4347BF583E527255BF55B7D49AF272C
:1020AF001227B3300121E54920E71C9079E07D49E3
:1020BF00AF271227B3AF27123B52EF700A200B073F
:1020CF007E3E7F0B1236A9E54954817047E527D331
:1020DF00940D400C200B3D7E3E7F1A1236A98034A2
:1020EF00E54BD394074028200B2A7E3E7F281236DB
:1020FF00A990756C7D49AF271227B37E757F6CE46D
:10210F00FBAD271238A47E3E7F341236A98005AF6F
:10211F002712321F300E2030001B907B08E0C39433
:10212F00645012055AE55A94F0400A90800074806A
:10213F00F0C2AF80FEC20E20020302224C9060015B
:10214F00E004F07006906000E004F0E5586031D3D1
:10215F009401400415588028907C20E004F0E0D3CF
:10216F009403400D200B077E3E7F361236A9124690
:10217F009E200B077E3E7F431236A9E4F558D22AE4
:10218F00302943E559703F907AF404F0A37408F0B6
:10219F00A37480F0A37401F0A37406F0907C0BE09D
:1021AF00907AF9F0907C0CE0907AFAF0907C0DE048
:1021BF00907AFBF0907C0EE0907AFCF0E4A3F0A311
:1021CF00F075590BC229302772907C09E07035E504
:1021DF00597031907AF47442F0A37408F0907C0A2D
:1021EF00E0907AF6F0907C0FE0907AF7F0A374010C
:1021FF00F0755906200B077E3E7F521236A9907C50
:10220F0009E004F0907C09E06402702FE559702B0F
:10221F00907AF47402F0A37408F0907C0AE0907A3C
:10222F00F6F0A3F0A37401F0755906200B077E3E5C
:10223F007F591236A9907C09E004F0C202122C4E8D
:02224F00C200CB
:01225100226A
:1045E600E55B602CE49078DDF0A3E55BF0907AE182
:1045F600E09078DFF0A37419F0907B0963A2019034
:1046060078E163A201AF5B1227C5E4F55B7F012267
:034616007F002200
:0B479C00302805C2287F01227F002288
:0100210022BC
:0647C100E4F55BF5472260
:0A47A700E490756CF0A3F0A3F0227B
:104619002043616E457247495400200A0045727271
:104629004C656E43616E21000A002043616E45723C
:0F46390072434821000A205265714572722100B8
:1030C700E59B541F6020200B1A7E467F191236A9F4
:1030D700E59B541FFF7E007D031237AA7E467F23A0
:1030E7001236A9E4F59BE5BA30E010E4F5B375B103
:1030F70080F5B2D22AF558907C20F0E5CFF4700322
:1031070002321C752901E4F528E5CFF4552970032F
:1031170002320AE528C454F0F5B1E5B2547F6420C1
:1031270060030231DBE5B3540FF54D85BC49E5BDBE
:10313700541FFF131313541FFFE5BD54E044184FEA
:10314700F54AE5BDC43354E0FFE5BE131313541F1E
:103157004FF54BE5BEC43354E0FFE5BF13131354DB
:103167001F4FF54C85A34E85A34F85A35085A351CB
:1031770085A35285A35385A35485A355E4F5B220AF
:10318700100CE549547EB5490575B350800375B3F6
:10319700D0E54D700AE549547EB549037F002230DA
:1031A7001008E54930E7037F0022E54DD394084036
:1031B7001D200B177E467F261236A9AF4D7E007D58
:1031C700031237AA7E467F311236A97F0022E54DCA
:1031D7002405FF22E5B2549F6023200B207E467F03
:1031E700331236A9AFB27E007D031237AAAFB37E82
:1031F700007D031237AA7E467F311236A9E4F5B265
:1032070075B3D0E52925E0F5290528E528C39408F5
:0732170050030231107F009B
:01321E00228D
:10432F00907B08E0C39464505675B180E4F5B3F503
:10433F00B28549BCE54BC4135407FFE54A54E04F1F
:10434F00F5BDE54B33333354F8FFE54CC413540735
:10435F004FF5BEE54C33333354F8F5BF854EA38587
:10436F004FA38550A38551A38552A38553A385548D
:10437F00A38555A3E54D540F2450F5B375580AC2C4
:02438F002A22E0
:1043910075B190E5B220E613200B107E467F3E12E8
:1043A10036A9AFB27E007D031237AAE4F5B3F5B2A8
:1043B1007472250FF582E43461F583E0F5BCE4F510
:1043C100BD7473250FF582E43461F583E0FF333367
:1043D1003354F8F5BE75BF78050F050F7472250FBC
:1043E100F582E43461F583E07002F50F75B3502274
:0947B100EF6003C29622D29622A9
:1042670043AB01C2E8C2EAE4FFEFC454F0F5B1C3BF
:10427700EF64809488500575B3D08003E4F5B3E408
:10428700F5B2F5BCF5BDF5BEF5BFF5C4F5C5F5C688
:10429700F5C7F5A3F5A3F5A3F5A3F5A3F5A3F5A333
:1042A700F5A30FBF0EC3907B08E0FF25E0F5B475BB
:1042B700B50C75B66C75A11275AB0275C13E75C3A9
:0442C700FF75C203BA
:0142CB0022D0
:100EC9005452414E5A004D41584200525453004425
:100ED900454C4159004E4F4B5654004B5000424F20
:100EE9004F540043414E004E4557504B5400415416
:100EF900004443440043414E4D4F4E0054454C3A43
:100F0900004C434C004454420054524300003E2AD2
:100F19002C312CCFE0F0E0ECE5F2F0FB20F3EFF020
:100F2900E0E2EBFFFEF9E5E3EE20EAEEEDF2F0EEAA
:100F3900EBEBE5F0E020CACF20C8F1E5F2FC0A00AE
:100F49003E4C2C6B30312C25732C43EAEEF0EEF13C
:100F5900F2FC20EDE020F8E8EDE52043414E2C308D
:100F6900202D20353030EAE1283530EC292C31208C
:100F79002D203530EAE128353030EC290A003020BF
:100F89002D20353030EAE1283530EC290031202D8B
:100F9900203530EAE128353030EC29003E532C6BFE
:100FA90030322C2562752CCCE0EAF12E20E0E4F0F9
:100FB900E5F120E1EBEEEAE020D2D128302D382905
:100FC9000A003E532C6B30332C2562752CCCE0EA99
:100FD900F12E20E0E4F0E5F120E1EBEEEAE020D2A9
:100FE900C8D228302D38290A003E532C6B30342CB6
:100FF9002562752CCCE0EAF12E20E0E4F0E5F12041
:10100900E1EBEEEAE020D2D328302D38290A003E60
:10101900422C6330312C2562752CC2F2EEF0E8F7D0
:10102900EDFBE920EAEEEDF2F0EEEBEBE5F020ED79
:10103900E020F8E8EDE50A003E2A2C312CCFE0F05B
:10104900E0ECE5F2F0FB20EFF0EEF2EEEAEEEBE099
:1010590020C8F1E5F2FC20EFEE20EFEEF0F2F320EC
:1010690052533233320A003E4C2C6B30352C256CEE
:10107900752CD1EAEEF0EEF1F2FC20EEE1ECE5EDB3
:10108900E020EDE020EFEEF0F2F32C3130302C329D
:1010990030302C3330302C3630302C313230302C4B
:1010A900323430302C343830302C393630302C3121
:1010B900393230302C33383430302C353736303003
:1010C9002C3131353230300A003E532C6B30362CFE
:1010D9002562752CCAEEEB2DE2EE20E1EBEEEAEE8D
:1010E900E220E220EFE0EAE5F2E50A003E422C6B5D
:1010F90030392C2562752CCDE520EFE5F0E5E4E0EB
:10110900E2E0F2FC20E4E8E0E3EDEEF1F2E8EAF3F4
:101119000A003E422C6B31302C2562752CD0E5F14A
:10112900F2E0F0F220EFF0E820EEF2F1F3F2F1F262
:10113900E2E8E820EFE5F0E5E4E0F7E820EFE0EAAF
:10114900E5F2EEE2203220ECE8ED2E0A003C210027
:101159003C6B30313D003C6B30323D003C6B3033F1
:101169003D003C6B30343D003C6330313D003C6B0D
:1011790030353D003C6B30363D003C6B30393D002D
:101189003C6B31303D0043796354530A004D65731C
:10119900730A00435449490A00435449540A005305
:1011A900705449540A0054696D655449540A000A37
:1011B9004173796E634F55543A00CEF820E4EBE859
:1011C900EDFB210A000A435243204552523A2000BE
:1011D9000A494E3A000A4173796E63494E3A003F13
:1011E9003F3F0A000089129B24AD36BF48C15AD33C
:1011F9006CE57EF78108931AA52CB73EC940DB52EE
:10120900ED64FF76028B109926AF34BD4AC358D1DD
:101219006EE77CF5830A9118A72EB53CCB42D950CD
:10122900EF66FD74048D169F20A932BB4CC55ED7AD
:1012390068E17AF3850C971EA128B33ACD44DF56AD
:10124900E960FB72068F149D22AB30B94EC75CD59D
:101259006AE378F1870E951CA32AB138CF46DD548D
:10126900EB62F97008811A932CA53EB740C952DB8D
:1012790064ED76FF89009B12AD24BF36C148D35A6D
:10128900E56CF77E0A8318912EA73CB542CB50D95D
:1012990066EF74FD8B029910AF26BD34C34AD1584D
:1012A900E76EF57C0C851E9728A13AB344CD56DF2D
:1012B90060E972FB8D049F16A920BB32C54CD75E2D
:1012C900E168F37A0E871C952AA338B146CF54DD1D
:1012D90062EB70F98F069D14AB22B930C74ED55C0D
:1012E900E36AF17800112332465765748C9DAFBECD
:1012F900CADBE9F810013322564775649C8DBFAEED
:10130900DACBF9E82130021367764455ADBC8E9FDC
:10131900EBFAC8D93120120377665445BDAC9E8FCC
:10132900FBEAD8C94253617004152736CEDFEDFCBC
:101339008899ABBA5243716014053726DECFFDECAC
:101349009889BBAA6372405125340617EFFECCDD9C
:10135900A9B88A9B7362504135241607FFEEDCCD8C
:10136900B9A89A8B8495A7B6C2D3E1F008192B3A8C
:101379004E5F6D7C9485B7A6D2C3F1E018093B2A6C
:101389005E4F7D6CA5B48697E3F2C0D129380A1B5C
:101399006F7E4C5DB5A49687F3E2D0C139281A0B4C
:1013A9007F6E5C4DC6D7E5F48091A3B24A5B69783C
:1013B9000C1D2F3ED6C7F5E49081B3A25A4B79682C
:1013C9001C0D3F2EE7F6C4D5A1B082936B7A48591C
:1013D9002D3C0E1FF7E6D4C5B1A092837B6A58490C
:1013E9003D2C1E0FFF0EC9FF0ECFFF0ED4FF0ED8E6
:1013F900FF0EDEFF0EE4FF0EE7FF0EECFF0EF0FF1F
:101409000EF7FF0EFAFF0EFEFF0F05FF0F0AFF0F83
:071419000EFF0F12FF0F167A
:0300230002337332
:0D337300C0E0C0F0C083C082C0D075D0188B
:1033800030984EC298750B01AF9920110FEF64026F
:10339000703F90616CF0D211D2918035301807C225
:1033A00018531F0F801CBF0904D2188024BF0312BA
:1033B00085636E636380536380C211750B00C29195
:1033C000800F74222563F582E4346FF583EFF005F6
:1033D000632099030234932012030234913017784A
:1033E000E56AB4FF0D759902056A756F00D2900207
:1033F0003491E56AB56214759903056A906F1FE010
:1034000070030234917401F0023491E56AD395623D
:10341000400DC212D21DC290E4FF1247B18072E586
:103420006F6009F599056A756F0080657422256AD9
:10343000F582E43470F583E0F56F6402600BE56FAC
:1034400064036005E56FB409057599098043856FCC
:1034500099056A756F0080397422256AF582E43413
:1034600070F583E0FF7008C212D21DC2908022D294
:1034700090C21DEFB47C09056A750832C212801132
:10348000AF6A056A74222FF582E43470F583E0F5A3
:0334900099C29945
:0B349300D0D0D082D083D0F0D0E03247
:103A7E007BFF7A0F791712198B907B08E070147503
:103A8E002FFF75300F7531877BFF7A0F7949121929
:103A9E008B8012752FFF75300F7531967BFF7A0F65
:103AAE00794912198B7BFF7A0F79A5906171E0F538
:103ABE002F12198B7BFF7A0F79CB90616BE0F52F6C
:103ACE0012198B7BFF7A0F79F2906102E0F52F12BB
:103ADE00198B7BFF7A107918A210E433F52F121987
:103AEE008B7BFF7A10794112198B907463E0FEA3E1
:103AFE00E0FFC3E49FFFE49EFEAB07FAE4F9F8FF94
:103B0E007E8C7D0AFC1222EA8F328E318D308C2F04
:103B1E007BFF7A10797012198B7BFF7A1079D28520
:103B2E006B2F12198B7BFF7A1079F5A219E433F5FE
:103B3E002F12198B7BFF7A11791B906F1FE0F52FD7
:043B4E0012198B229B
:10349E007E117F56123EECEF4E70037F0122E490B8
:1034AE007B08F07E117F59123EECEF4E60151247ED
:1034BE0046BF3106907B08740AF0BF3206907B0837
:1034CE007464F07E117F5F123EECEF4E6008124383
:1034DE00F1906171EFF07E117F65123EECEF4E6060
:1034EE00081243F190616BEFF07E117F6B123EEC90
:1034FE00EF4E60081243F1906102EFF07E117F7182
:10350E00123EECEF4E600D1243F1EC4D4E4F24FF88
:10351E0092108002C2107E117F77123EECEF4E6049
:10352E00231243F1A804A905AA06AB077F007E8CDF
:10353E007D0A7C001222EA12237C907463EEF0A3C3
:10354E00EFF0800A90746374FFF0A374DCF07E11C8
:10355E007F7D123EECEF4E60071243F18F6B8003BE
:10356E00756B02E56B7003756B017E117F83123EE6
:10357E00ECEF4E600A124746EF24D024FF92197EDC
:10358E00117F89123EECEF4E600A124746EF24D0AF
:06359E00906F1FF07F009A
:0135A4002204
:1028D300E4F50F907C34F0907C34E075F003A4248D
:1028E300EDF582E43413F583E493FB740193FA74F6
:1028F3000293F91222527003022AA9E4907C36F063
:10290300A3F0907C35F0907C35E02494F582E43498
:1029130075F583E0FF7003022AA0907C34E075F024
:1029230003A424EDF582E43413F583E493FB7401EB
:1029330093FA740293F9907C36E0F5827583001262
:10294300226BFEEFB5060F907C377401F0907C3656
:10295300E004F0022A97907C37E07003022A97EE96
:102963006003022A8E907C34E014607424FC7003AC
:10297300022A50147003022A7E147003022A2024B0
:10298300F97003022A82147003022A86240F60035B
:10299300022AA0907C35E02494F9E43475FA7B0193
:1029A300C0031B8B2F753000753100E4F532D00363
:1029B300122AAA907C3812239B907C38E0F8A3E07B
:1029C300F9A3E0FAA3E0FB7F007E8C7D0A7C001272
:1029D30022EA12237C907463EEF0A3EFF0022AA0A4
:1029E300907C35E0FD2494F582E43475F583E0248E
:1029F300D0906171F074952DF582E43475F583E020
:102A030024D090616BF0907C35E02496F582E43419
:102A130075F583E024D0906102F0022AA0907C3502
:102A2300E02494F9E43475FA7B01C0031B8B2F7502
:102A33003000753100E4F532D003122AAA907C38B5
:102A430012239B907C3BE0907B08F08050907C3578
:102A5300E02494F9E43475FA7B01C0031B8B2F75D2
:102A63003000753100E4F532D003122AAA907C3885
:102A730012239B907C3BE0F56D8022D213801ED203
:102A830019801A906F1F7401F08012E4907C37F064
:102A9300907C36F0907C35E004F0022909907C3478
:062AA300E004F00228DA55
:012AA900220A
:1024E500E4906170F09061B5F0C21690616EF09065
:1024F5006F1E7405F0C212C21DC211C218E4F56A3E
:10250500F562F508F563F50B90746374FFF0A37439
:10251500F4F09061027402F090616BF0906171F0DB
:10252500C21BD21AC210907122741EF0E4907B086F
:10253500F0C213C215C214F56DC219906F1FF0D207
:102545001712349EEF60031228D3907122E0049095
:10255500616DF0E4F50F907C327461F0A37472F054
:10256500906171E0F50FE50FC394014007E50FD3C6
:1025750094084003E4F50FE50F6028907C32E4757C
:10258500F00112229885F082F58374C4F0150F903E
:102595007C32E475F00112229885F082F583E50F0F
:1025A500F080D490616BE0F50FE50FC3940140070F
:1025B500E50FD394084003E4F50FE50F6028907C00
:1025C50032E475F00112229885F082F58374C8F023
:1025D500150F907C32E475F00112229885F082F592
:1025E50083E50FF080D4906102E0F50FE50FC39409
:1025F500014007E50FD394084003E4F50FE50F60AC
:1026050028907C32E475F00112229885F082F583DA
:1026150074C2F0150F907C32E475F0011222988592
:10262500F082F583E50FF080D4907C32E475F001FB
:1026350012229885F082F583E4F0907C3275F001E2
:1026450012229885F082F583E4F0F50FF56C75F0AC
:1026550075E56CA42436F582E5F03468F583E4F07D
:10266500E56C75F00DA42403F582E43461F583E48B
:10267500F0F56175F068E56CA42423F582E5F03486
:1026850071F58375F00DE5611223D8E4F00561E578
:1026950061B408DF056CE56CB408B3E4F571F55D6C
:1026A500F55FF560F569F570F561F55EF56CF56852
:1026B500C2ADF5C9D2CDD2CCC2C9C2CAF5CDF5CC11
:1026C500907463E0F5CBA3E0F5CA85CBCD85CACC84
:1026D500D29ED29CD2CAC2ACC298C29975B81075A6
:0426E500B710D2ACAC
:0126E90022CE
:0100220022BB
:10321F008F2830190EE549B44209E54C640270035A
:10322F00023372E54A54E324DF606D24DF604214F9
:10323F00603F24E370030232CE1470030233201474
:10324F00700302335124E26028246060030233725A
:10325F00300C077E117F8F1236A9E54B75F00DA448
:10326F002403F582E43461F5837D49AF281227B337
:10327F0022300C077E117F961236A975F00DE5608E
:10328F00A424DEF582E5F0346BF5837D49AF281277
:10329F0027B3056053603F22300C077E117F9C12CD
:1032AF0036A975F00DE55DA424B6F582E5F034611D
:1032BF00F5837D49AF281227B3055D535D7F22301B
:1032CF000C077E117FA21236A975F075E54BA42469
:1032DF0043F582E5F03468F583E54C541FFF131373
:1032EF00543F75F00D1223D87D49AF281227B375BF
:1032FF00F068E54BA42423F582E5F03471F583E5FE
:10330F004C541FFF1313543F75F00D1223D8E4F0E4
:10331F0022300C077E117FA81236A975F068E54B95
:10332F00A42423F582E5F03471F583E54C543FFF77
:10333F001313543F75F00D1223D87D497F0D1227BB
:10334F00B322300C077E117FAF1236A975F075E5E9
:10335F004BA42436F582E5F03468F5837D49AF2818
:04336F001227B3224C
:103D38008F2B90600263A20190702263A201AF2BC7
:103D48001227C5E4F564F565852B6790702263A298
:103D5800019011ED63A201AF67AE66AD65AC641268
:103D680028018F678E668D658C647422252BF582F9
:103D7800E43470F583E565F07423252BF582E4348B
:103D880070F583E564F07422252BF582E43470F530
:103D980083E0FFA3E0906F20CFF0A3EFF0E52B24A2
:103DA80002F562200B127E117FB81236A97E707F51
:103DB80022E4FBAD621238A47F011247B1756AFF95
:0A3DC800D212C2992099FDD299226F
:101C8500E560655F605875F00DE55FA424E2F582B7
:101C9500E5F0346BF583E02405F52BD3940E400C69
:101CA500200B357E117FC31236A9802C75F00DE50A
:101CB5005FA424DEF582E5F0346BF58363A201743D
:101CC500042568F582E43460F58363A201AF2B1225
:101CD50027C5E52B2568F568055F535F3F2275F03D
:101CE50075E56CA42436F582E5F03468F583E0707B
:101CF50003021DECE55E705575F075E56CA4243A9C
:101D0500F582E5F03468F583E02405F52BD3940ED0
:101D1500400C200B357E117FC31236A9802C75F03F
:101D250075E56CA42436F582E5F03468F58363A285
:101D35000174042568F582E43460F58363A201AF7C
:101D45002B1227C5E52B2568F568055E2275F0750C
:101D5500E56CA42439F582E5F03468F583E0540F89
:101D6500FFE55ED39F506575F075E56CA4243AF5E3
:101D750082E5F03468F58375F00DE55E1223D8E051
:101D85002405F52BD3940E400C200B3D7E117FC30B
:101D95001236A9803475F075E56CA42436F582E514
:101DA500F03468F58375F00DE55E1223D863A20162
:101DB50074042568F582E43460F58363A201AF2BD2
:101DC5001227C5E52B2568F568055E22E4F55E75E5
:101DD500F075E56CA42436F582E5F03468F583E406
:101DE500F0056C536C0722056C536C07E55D657156
:101DF500605875F00DE571A424BAF582E5F03461FB
:101E0500F583E02405F52BD3940E400C200B357E8D
:101E1500117FC31236A9802C75F00DE571A424B687
:101E2500F582E5F03461F58363A20174042568F554
:101E350082E43460F58363A201AF2B1227C5E52B3D
:101E45002568F568057153717F22E56975F00DA464
:101E55002403F582E43461F583E06067E56975F094
:101E65000DA42407F582E43461F583E02405F52B00
:101E7500D3940E400C200B347E117FC31236A980FB
:101E85002BE56975F00DA42403F582E43461F5832F
:101E950063A20174042568F582E43460F58363A2C6
:101EA50001AF2B1227C5E52B2568F568E56975F0A7
:101EB5000DA42403F582E43461F583E4F005695348
:101EC500690722056953690775F068E570A424233D
:101ED500F582E5F03471F58375F00DE5611223D8CF
:101EE500E07003021F6D75F068E570A42427F58284
:101EF500E5F03471F58375F00DE5611223D8E02422
:101F050005F52BD3940E400C200B3D7E117FC3129B
:101F150036A9803475F068E570A42423F582E5F0D0
:101F25003471F58375F00DE5611223D863A2017450
:101F3500042568F582E43460F58363A201AF2B12B2
:101F450027C5E52B2568F56875F068E570A4242399
:101F5500F582E5F03471F58375F00DE5611223D84E
:101F6500E4F00561536107220561E561C39408400A
:091F750008E4F5610570537007E2
:011F7E002240
:102C4E00300028C200906F1FE0601204F0E0D394B1
:102C5E00F0400A9080007480F0C2AF80FE90616FE9
:102C6E00E004F09061B5E0600214F0E508B4010CE8
:102C7E00E4F508D212C2992099FDD299E50BD394AE
:102C8E00644007C211E4F563F50B30120F90616FCB
:102C9E00E0D39414400BC212D21D8005E490616FF4
:102CAE00F020123EE508703A301A37F528E528C3B1
:102CBE00956B5010121C85E5686009D394C85004BA
:102CCE00052880E9E568601AE4906002F0A37419A3
:102CDE00F0E5682402FF123D38E4F568906000F0DC
:102CEE00A3F0E56E7003022DEBF528E4F56EF564A6
:102CFE00F565E528547FF567E52854802422F58292
:102D0E00E4346FF58363A2019011ED63A201AF6706
:102D1E00AE66AD65AC641228018F678E668D658CCC
:102D2E0064E52854802422F582E4346FAF82F529BD
:102D3E008F2A53287FE56545646022300B03022DF0
:102D4E00EB7E117FCE1236A9E4FBAD28AF2AAE2959
:102D5E001238A47D03AF65AE641237AA22200B2E63
:102D6E00906170E0640160147E117FD91236A9E47F
:102D7E00FBAD28AF2AAE291238A480127E117FDE59
:102D8E001236A9E4FBAD28AF2AAE291238A4E528E5
:102D9E00B40408E490616DF0C21C22852A82852954
:102DAE0083A3E024E7702CD216E52824FCF559C342
:102DBE00940E501BE52A2402FFE43529F5838F82F9
:102DCE0063A201907AF463A201AF591227C522E4DF
:0D2DDE00F55922200B077E117FE81236A95F
:012DEB0022C5
:103E6C000208A4E493A3F8E493A34003F68001F2C0
:103E7C0008DFF48029E493A3F85407240CC8C33357
:103E8C00C4540F4420C8834004F456800146F6DF26
:103E9C00E4800B01020408102040809047BAE47EB5
:103EAC00019360BCA3FF543F30E509541FFEE4931B
:103EBC00A360010ECF54C025E060A840B8E493A3E2
:103ECC00FAE493A3F8E493A3C8C582C8CAC583CA0D
:103EDC00F0A3C8C582C8CAC583CADFE9DEE780BEC5
:0147C00000F8
:10225200BB010689828A83E0225002E722BBFE028A
:09226200E32289828A83E49322BD
:10226B00BB010CE58229F582E5833AF583E0225028
:10227B0006E92582F8E622BBFE06E92582F8E22272
:0D228B00E58229F582E5833AF583E493228C
:10229800A3F8E0C5F025F0F0E582158270021583F9
:0622A800E0C838F0E82256
:1022AE0075F008758200EF2FFFEE33FECD33CDCCE7
:1022BE0033CCC58233C5829BED9AEC99E58298406A
:1022CE000CF582EE9BFEED9AFDEC99FC0FD5F0D647
:1022DE00E4CEFBE4CDFAE4CCF9A88222B800C1B971
:1022EE000059BA002DEC8BF084CFCECDFCE5F0CBAF
:1022FE00F97818EF2FFFEE33FEED33FDEC33FCEBE8
:10230E0033FB10D703994004EB99FB0FD8E5E4F9A2
:10231E00FA227818EF2FFFEE33FEED33FDEC33FC8F
:10232E00C933C910D7059BE99A4007EC9BFCE99A83
:10233E00F90FD8E0E4C9FAE4CCFB2275F010EF2FC8
:10234E00FFEE33FEED33FDCC33CCC833C810D707C8
:10235E009BEC9AE899400AED9BFDEC9AFCE899F803
:0E236E000FD5F0DAE4CDFBE4CCFAE4C8F92296
:0E237C00C3E49FFFE49EFEE49DFDE49CFC2272
:10238A00EB9FF5F0EA9E42F0E99D42F0E89C45F0A9
:01239A002220
:0C239B00ECF0A3EDF0A3EEF0A3EFF022B5
:1023A700A8828583F0D083D0821223BE1223BE1267
:1023B70023BE1223BEE473E493A3C583C5F0C5838C
:1023C700C8C582C8F0A3C583C5F0C583C8C582C880
:0123D70022E3
:0C23D800A42582F582E5F03583F5832210
:10192900E53B242FF8E6053B22782C302502782F59
:10193900E475F001122445022252201EEB7F2ED2BB
:101949001E8018EF540F2490D43440D4FF30220B5A
:10195900EF24BFB41A0050032461FFE53C6002156F
:101969003C053FE53F7002053E30250D782CE475B6
:10197900F001122445EF0223E40244A77403D2259F
:101989008003E4C225F53B8B2C8A2D892EE4F53C96
:10199900F53EF53FE53C60077F2012196480F57537
:1019A9003DFFC21FC21EC220C221C223C224C226B9
:1019B900121932FF700D3025057F00121975AF3FDE
:1019C900AE3E22B4255FC2D5C222121932FF24D0FD
:1019D900B40A00501A75F00A783C30D50508B6FFEC
:1019E9000106C6A426F620D5047002D22180D92486
:1019F900CFB41A00EF5004C2E5D222021B75D21FE0
:101A090080C6D21E80C0D22080BCD2D580BAD22353
:101A190080B47F201219642020077401B53C00406E
:101A2900F1121929FF12196402199DD226D22480B4
:101A390095121929FB121929FA121929F94A4B7019
:101A49000679467A1C7BFF20202EE53C602A7E0021
:101A59008E8275830012226B60060EEE653D70F072
:101A6900C2D5EBC0E0EAC0E0E9C0E0EE121BBCD091
:101A7900E0F9D0E0FAD0E0FB122252FF60AAEBC0F5
:101A8900E0EAC0E0E9C0E0121964D0E02401F9D02D
:101A9900E03400FAD0E0FBE53D0460DCD53DD980B7
:101AA900877BFF7A1B79B8D220809C7910800279D4
:101AB90008C224C2268008D2D5790A8004790AC2CC
:101AC900D5E53D047002F53DE4FAFDFEFF12192942
:101AD900FC7B08201F13121929FD7B10301E0A12E6
:101AE9001929FE121929FF7B20EC3382D592D55092
:101AF90013C3E4301E069FFFE49EFEE4201F039DEE
:101B0900FDE49CFCE4CBF8C21FEC700CCFCECDCC2D
:101B1900E824F8F870F38017C3EF33FFEE33FEEDD6
:101B290033FDEC33FCEB33FB994002FB0FD8E9EBB7
:101B3900301F05F8D0E0C448B21FC0E00AEC4D4E92
:101B49004F78207B0070C2EAB53D0040BCC0E0126E
:101B59001BBED0F0D0E0201F04C4C0E0C4B21FC037
:101B6900F012194DD0F0D5F0EB02199D1224A41AE8
:101B79003A531AB4581A0B4C1A07421AB84F1AC0DA
:0F1B8900441AC0491A20431AC6551AAA461AAA66
:101B9800451AAA471C66501A0F2D1A132E1A362BEF
:101BA8001A17231A34201C4F2A19CF4800001A2E5E
:101BB8003F3F3F00790AA2D5202114302309B910EC
:101BC800020404B9080104A2D5202402500104200B
:101BD80020689220B53C005034C0E07F20302119A5
:101BE8007F30A22072247223500F121C15C220C20B
:101BF80024C223C2267F30800F302303E9C0E012BD
:101C08001964302303D0E0F9D0E0B53CCC30231779
:101C18007F30B9100C1219647F583022077F788002
:101C280003B908031219643020057F2D0219647F57
:101C3800202026F87F2B2024F322922080CF286EA4
:101C4800756C6C2900D21F121929301FF8C21F7831
:101C58003C30D50108F60219CF2D504349581219C6
:101C6800292403B405004001E4901C61931219551E
:0D1C7800743A121955D221753C04021AB4B9
:102AAA008B2C8A2D892EE4F538F537F536F535F570
:102ABA0033F534E5304531452F6012EBC0E0EAC00A
:102ACA00E0E9C0E0AB2FAA30A931122455AB2C059E
:102ADA002EE52EAA2D7002052D14F9122252F5396F
:102AEA00C394094007E539D3940D40E1E5396420E0
:102AFA0060DBE539B42D054334038016E539B42B80
:102B0A0005433401800C74FF252EF52E74FF352DF4
:102B1A00F52DE53260046410703FAB2CAA2DA92E66
:102B2A0012225264306009E532702E75320A802909
:102B3A0090000112226BFF64786004EFB4581343CB
:102B4A0034017532107402252EF52EE4352DF52D3B
:102B5A008007E5327003753208AB2C052EE52EAAE4
:102B6A002D7002052D14F9122252F539C3946140D1
:102B7A000AE539D3947A50035339DF74D02539F5ED
:102B8A0039C3940A400CE5399411406D74F925391A
:102B9A00F539E539D39532506043340185383D859E
:102BAA00373C85363B85353AAF327E00E4FCFDABD7
:102BBA0038AA37A936A8351223F6C8ECC8C9EDC910
:102BCA00CAEECACBEFCBE4FCFDFEEB2539F538EEB5
:102BDA003AF537ED39F536EC38F535AF38AE37AD6D
:102BEA0036FCAB3DAA3CA93BA83AD312238A500330
:102BFA00022B63433404022B63E53420E003E480B0
:102C0A002DE5304531452F601EAB2CE52E24FFF90A
:102C1A00E52D34FFFAEBC0E0EAC0E0E9C0E0AB2FF3
:102C2A00AA30A931122455E53430E20774FFFFFEB9
:102C3A00FDFC22E534AF38AE37AD36AC3530E103B2
:042C4A0002237C22C3
:1023E400BB010689828A83F0225002F722BBFE01D8
:0223F400F322D2
:1023F600E88FF0A4CC8BF0A42CFCE98EF0A42CFC86
:102406008AF0EDA42CFCEA8EF0A4CDA8F08BF0A403
:102416002DCC3825F0FDE98FF0A42CCD35F0FCEB62
:102426008EF0A4FEA9F0EB8FF0A4CFC5F02ECD3927
:0F243600FEE43CFCEAA42DCE35F0FDE43CFC2294
:10244500FAE6FB0808E6F925F0F618E6CA3AF62298
:10245500BB011A89828A83D0F0D0E0F8D0E0F9D0A8
:10246500E0FAD0E0FBE8C0E0C0F00224D35016E962
:10247500F8D083D082D0E0F9D0E0FAD0E0FBC0827A
:10248500C0830224CABBFE16E9F8D083D082D0E00F
:0F249500F9D0E0FAD0E0FBC082C0830224DC2241
:1024A400D083D082F8E4937012740193700DA3A3C7
:1024B40093F8740193F5828883E4737402936860DB
:0624C400EFA3A3A380DFDB
:0924CA00EBF608EAF608E9F62237
:0924D300EBF0A3EAF0A3E9F0220A
:0924DC00EBF208EAF208E9F22231
:00000001FF
